:040000000C946803F1
:100004000C9400000C9400000C9400000C9400006C
:100014000C9400000C9400000C9400000C9400005C
:100024000C9400000C9400000C9400000C9400004C
:100034000C9400000C9400000C9400000C9400003C
:100044000C9400000C9400000C9400000C9400002C
:100054000C9400000C9400000C94A6030C94000073
:100064000C9400000C9400000C9400000C9400000C
:100074000C9400000C9400000C9400000C940000FC
:100084000C9400000C9400000C9400000C940000EC
:100094000C9400000C9400000C9400000C940000DC
:1000A4000C9400000C9400000C9400000C940000CC
:1000B4000C9400000C9400000C9400000C940000BC
:1000C4000C9400000C9400000C9400000C940000AC
:1000D4000C9400000C9400000C9400000C9400009C
:1000E40000FEFE000000000000000000000F0F0CE6
:1000F4000C0C0C0C0000000000FEFEE0B0180C0616
:1001040002000000000F0F000103060C08000000AD
:10011400003844444444380000FC000000001E122F
:1001240012121212121E000000FC4040FC4040FC5F
:1001340000FC0000000F08080F00001F001F000053
:1001440000FC04040404040000FC0000000F080880
:1001540008080808001F00000000FC8484848484CC
:100164008484000000080808080808080808080033
:10017400000404FC044440FC00FC0000000C0300E8
:10018400030C001F001F00000080A4A4BCA4A4BC96
:10019400A4A4800000001E1212121312121E0000EA
:1001A40000040404FC00FC8080FC0000000804033C
:1001B40000001F00001F0000007C484848487C00E5
:1001C400007C101000001D151515151515170000DD
:1001D40000F804040404F80000FC00000007080808
:1001E40008080700001F00000084848444245C483D
:1001F40048FC000000000C1212121212120C000033
:10020400007C40404040404000FC101000001E12A2
:1002140012121212121E00000000C0300C30C00076
:1002240000000000000E01010101010E00000000A9
:10023400001CE0000000E01C0000000000000003BF
:100244000C0300000000000000FC44444444B800D7
:1002540000000000000F000000000F00000000007C
:1002640000FC84848484780000000000000F0000F7
:1002740000000000000000000000000000FC00007E
:100284000000000000000000000F0000000000005B
:1002940000F008040404040800000000000304083B
:1002A400080808040000000000000000000000002E
:1002B4000000000000100800000000000000000022
:1002C40000FC84848484780000000000000F000097
:1002D40000000000000000000000C0300C30C0002E
:1002E40000000000000E01010101010E00000000E9
:1002F40000FC04040408F00000000000000F0808DB
:1003040008040300000000000038444484841800FA
:1003140000000000000608080808070000000000AC
:10032400000004C40404C40404FC00000008080F12
:1003340008080F080A090800008098A4A4A4A4A42B
:10034400A49880000000020302020202031E0000BF
:10035400000484641C24449410FC000000011C105C
:10036400101010101013000000003C242424242436
:10037400243C000000011D1111111711111101007D
:100384000084848444241C0000FC202000000C12FF
:1003940012121212120C0000000000807C80000077
:1003A40000FC80800008060100010608001F000010
:1003B400000484641C24449410FC000000011C10FC
:1003C4001010101010130000000404847C84040432
:1003D40000FC80800008060100010608001F0000E0
:1003E40000040404FC00FC8080FC000000080403FA
:1003F40000001F00001F0000007C484848487C00A3
:10040400007C101000001D1515151515151700009A
:10041400008098E4A4A4A4A4E498800000000C1232
:1004240012121212120C00000038444444443828BA
:1004340028FC00000000020202020202021E000068
:1004440000FC04040404FC0000FC8080000F080885
:1004540008080F00001F000000F804040404F8005A
:1004640000FC00000007080808080700001F00003F
:100474000094949454341C1010FC000000001E12CC
:1004840012121212121E0000000404FC044440FC68
:1004940000FC0000000C0300030C001F001F000000
:1004A40000F804040404F84040FC000000070808B5
:1004B40008080700001F0000000080601C20408026
:1004C40000FC000000011C1010101010101300009C
:1004D400000404FC044440FC00FC0000000C030085
:1004E400030C001F001F00000080A4A4BCA4A4BC33
:1004F400A4A4800000001E1212121312121E000087
:1005040000040404FC00FC8080FC000000080403D8
:1005140000001F00001F0000007C484848487C0081
:10052400007C101000001D15151515151517000079
:1005340000FC44444444B80000000000000F0000E4
:1005440000000F000000000000FC186080008060C4
:1005540018FC0000000F000001060100000F00005D
:10056400001090545454901000FC00000008090A34
:100574000E0A0908001F00000000E4242424242497
:10058400243C00000008090909090F0909090800A9
:10059400008040301C205010107C000000001D150D
:1005A400151515151517000000040404FC1010FCA3
:1005B40000FC0000000804030001011F001F0000EC
:1005C400008484FC84FC849410FC000000001E124F
:1005D40012121212121E000000384444443800FC67
:1005E40000FC0000000109070105041F001F0000B2
:1005F40000F804040404F84040FC00000007080864
:1006040008080700001F000000FC8484848478002C
:1006140000000000000F00000000000000000000C7
:1006240000F00804040404080000000000030408A7
:10063400080808040000000000FC44444444B800D6
:1006440000000000000F0808080807000000000070
:1006540000E01804000000000000000000030C107B
:100664000000000000000000000418E0000000008A
:100674000000000000100C03000000000000000057
:100684000000FC909090909090FC000000080808F6
:1006940008080F08080808000000FC848484848487
:1006A40084840000000808080808080808080800EE
:1006B4001027E80364000A00010000100001100084
:1006C4000100000001000400C6060000F894EE27B3
:1006D400EFBBF1E0F5BFE5BFE0937400E093750074
:1006E400F8E1A895A4B7A77FA4BFF0936000E093B6
:1006F40060008DE0A2E0BB27ED938A95E9F780E0E6
:1007040090E2A0E0B2E0ED930197E9F7E8ECF6E0BF
:1007140085919591009761F0A591B59105901590FB
:10072400BF01F00105900D920197E1F7FB01F0CFB5
:100734008BBF8CBFE0E0EEBBEFEFEDBFE1E2EEBFBD
:10074400C0E0D6E00C94D305AA93BA93EA93FA9343
:10075400EFB7EA93A4E0B6E0ED91FD913196FE93F4
:10076400EE93A0910406B0910506A83EE3E0BE070F
:1007740098F04394A0E0F399A1E0E1E0EA2711F4B2
:10078400F39801C0F39AE0E0E0930406E0930506D1
:10079400EAE04E1608F04424E991EFBFF991E9919B
:1007A400B991A991189580EA8A95F1F7589AE88148
:1007B400E8B95A9A000008C080EA8A95F1F7589877
:1007C400E881E8B95A9A00005A98219608955C9AEB
:1007D4005D9AEFE3EA93F0DFE0EC17C0E0E4E09326
:1007E4000106F1980895E0E4E0930106F19A089572
:1007F400F19B03C05C985D9A02C05C9A5D98E0919D
:100804000206EA93D9DFE0910106EA93D5DF089561
:100814001A93EEDFE0E0E0930006F29B02C00E9430
:10082400EA0510E0E9811E1720F40E94F0051F5F1D
:10083400F9CF0E94F505E0E0E0930006F29B07C0C3
:100844000E94EA05E0910006EF77E093000610E0CD
:10085400E9811E1720F40E94F0051F5FF9CFE09193
:100864000106A981EA0F0E94FC05188122960895C9
:100874000E948006EC81ACE0EA02002DB9DF10E0B2
:10088400101750F40E940306F29B02C00E94EA056E
:100894000E94F0051F5FF4CFE02FEE0F3E2F0E9461
:1008A400F505102F131778F40E940306F29B07C076
:1008B4000E94EA05E0910006EF77E09300060E94AB
:1008C400F0051F5FEFCFE0910106E00F0E94FC05E9
:1008D4000E9485062796089581DF0E940D060E94D6
:1008E4001406E4EEF0E00E941806ECEFF0E00E943B
:1008F4001806E4E1F1E00E94180675DF0E940D0677
:10090400ECE2F1E00E941806E4E4F1E00E9418062B
:10091400ECE5F1E00E9418060E9414060895E42D07
:10092400F0E0309711F50E941E06E4EBF3E00E941C
:100934001806ECECF3E00E941806E4EEF3E00E94E3
:100944001806ECEFF3E00E9418060E942A06E4E180
:10095400F4E00E941806ECE2F4E00E9418060E94FB
:1009640033060E943606E0E12DC0E530A0E0FA0728
:1009740059F50E941E06E4E4F4E00E941806ECE532
:10098400F4E00E941806E4E7F4E00E941806ECE89C
:10099400F4E00E9418060E942A06E4EAF4E00E94A9
:1009A4001806E4E8F6E00E941806ECE9F6E00E9476
:1009B4001806E4E0F5E00E941806ECE1F5E00E9478
:1009C4001806E3E0EA9324DF0895E42DF0E030977D
:1009D400F9F40E943906ECE1F2E00E941806E4E31F
:1009E400F2E00E941806ECE4F2E00E9418060E946D
:1009F40045060E9448060E944B060E9433060E9448
:100A040036060E9456060E9459060E945C0696C04D
:100A1400E230A0E0FA07F9F40E943906E4E6F2E0D5
:100A24000E941806ECE7F2E00E941806E4E9F2E0FE
:100A34000E9418060E9445060E9448060E944B0622
:100A44000E9433060E9436060E9456060E945906EA
:100A54000E945C0673C0E430A0E0FA07F9F40E9437
:100A64003906ECEDF2E00E941806E4E3F5E00E949A
:100A74001806ECE4F5E00E9418060E9445060E9460
:100A840048060E944B060E9433060E9436060E94C6
:100A940056060E9459060E945C0650C0E630A0E04B
:100AA400FA0721F50E943906ECE0F6E00E941806E8
:100AB400E4E2F6E00E941806ECE3F6E00E94180671
:100AC400E4E9F5E00E941806ECEAF5E00E94180655
:100AD4000E9460060E9433060E9436060E94560653
:100AE4000E945906EFE0EA9393DE28C0E830A0E0C4
:100AF400FA0721F50E943906E4EBF3E00E94180698
:100B0400ECECF3E00E941806E4E6F5E00E94180617
:100B1400ECE7F5E00E941806E4E9F5E00E94180607
:100B24000E946006ECEAF5E00E9418060E94330673
:100B34000E9436060E9456060E9459060895E0E077
:100B4400F399E1E0E03069F40E946906F29A0E94A8
:100B54007106ECEEF1E00E9418060E947806F29A03
:100B64000EC0E130E9F40E946906F2980E94710611
:100B7400ECEEF1E00E9418060E947806F298E4E098
:100B8400F2E00E941806E1E0EA9342DEE4E8F3E0D2
:100B94000E941806ECE9F3E00E9418060E9414066D
:100BA4000895EFEFE7B9EAB95E9AEFE05E2EE0E070
:100BB400E4BDE3E0E5BDE6E0E6BDE1E0E0936E0020
:100BC40006DE789489DEABDEBADFFFDEFBCFFFCF33
:100BD400E0910006E095E09300060895E091000698
:100BE400EA930C94D503E0910206EF5FE0930206CA
:100BF4000C94FA03E0930106E0910306E0930206E5
:100C04000895E12FAD81BE81F0E0EA0FFB1F04904F
:100C1400009200060895E8EBE0930206E0930306D1
:100C2400F29A0895ECE1EA930C940A04FA93EA9395
:100C3400E1E0EA930C943A040E94F003EAEBE093B7
:100C44000206E0930306F298E0E1EA930C940A04A6
:100C54000E94F503EAEBE0930206E0930306F298A0
:100C64000895E4E5F3E0E2CFECE6F3E0DFCF0E94A1
:100C7400F003ECEBE0930206E0930306F29AE4E05F
:100C8400EA930C940A04E4ECF5E0D0CFECEDF5E043
:100C9400CDCF0E94F503ECEBE0930206E09303064C
:100CA400F29AE4EFF5E0C2CFE4E2F3E0BFCFECE385
:100CB400F3E0BCCFE5E0EA930C940A040E94F50348
:100CC400ECEBE0930206E0930306F29A08950E9487
:100CD400F003EEEBE0930206E09303060895E8E2E6
:100CE400EA930E940A04E4EDF1E0A0CF0E94F50328
:100CF400EEEBE0930206E093030608953A932A93F9
:100D04001A930A9308953B812A81198108810895D1
:00000001FF
